:020000040000FA
:020000001D28B9
:08000800F000030EF100831269
:10001000F33086058316730892008312741F172825
:10002000221C15280000061516288615A20A8C0128
:10003000710E8300F00E700E0900830107309F00DF
:100040008B0186016400F401F50183169F01810193
:10005000D0308600EF3085008312C830A500222101
:10006000A50B2F286430A500F4172221A50B3428F6
:1000700083169B011C141A08F200523C03184328F3
:100080005230F20049283C30720203185A283C30A2
:10009000F20083168B01F401F5019B0172089A00AE
:1000A0001C1555309D00AA309D009C1464009C18BE
:1000B00056281C1183120A30A500F401F501C8303E
:1000C000A100043092002221A50B5D280530A50077
:1000D000F401F501F4172221A50B68288C0185187D
:1000E0005A281E30A5007208F300831602308C00D7
:1000F0008312C830A10085185A28C0308B007510B3
:100100007417F417061E88282221A50B732832289D
:100110007514831602308C008101E7308500D030E1
:1001200086009B011C141A08F200831286166400D4
:10013000CA309F00831680309F0083120130A000D8
:100140001A21061A71289F1BAD2883169F0A831255
:10015000A00A2008103C0318A028A00307309F0025
:1001600083169F018312F417200821020319C42863
:100170002221061A71282221061A71282008A100BE
:100180000310200D7202F300C830A5003921741C41
:100190000029F41D0029F4132221061A7128A50B49
:1001A000C628F4172221F41CD128741ED128F4107B
:1001B0007412F41722217208F3003230A600F413EF
:1001C0002221F41CE628741EE628ED28F4180821E4
:1001D000741A1121A60BDF28D928F41774132221D1
:1001E00022212221222122212221222122212221F7
:1001F00022212221222122212221222122214928B9
:10020000C0308B00741785181D28061A712888289D
:10021000F410F2033C307202031808003C30F20084
:1002200008007412F20A7208523C03180800523097
:10023000F2000800A40164000516061A0800A40BC9
:100240001B2908000730A3001E30A4006400751CA1
:100250002B29061A08000B1D26290B11A30B262992
:100260000730A300F41B3629051637290512A40B05
:100270002629861F7414061FF415861F0800061F02
:100280000800741C4B29741948297415F4104B2963
:1002900074107411F414F41D0800F41A5229F416A1
:0C02A00074120800F411F4127416080027
:02400E00463F2B
:00000001FF
